:020000000628D0
:10000800803109008801F32B2000B301BB234D2365
:100018002000AF00AF362F08483A031DD028210032
:100028008E1220000E1E15280E1A182821008E1672
:100038004D232000AD002D03031DCB2821008E1277
:1000480020000E1E24280E1A272821008E164D2364
:100058002000AE003206031DC62821008E122000A3
:100068000E1E33280E1A362821008E164D23200026
:10007800B10021008E1220000E1E3F280E1A4228C1
:1000880021008E1620003108213A031D4D284C21ED
:10009800C3283108043A031D5F284D232000B0000F
:1000A80021008E1220000E1E56280E1A59282100F3
:1000B8008E16043095283108B03A031D71284D2357
:1000C8002000B00021008E1220000E1E68280E1A93
:1000D8006B2821008E160B3095283103031D8428C8
:1000E8004D232000B00021008E1220000E1E79281A
:1000F8000E1A7C2821008E162000B301B30AC328EB
:100108003108023A031D98284D232000B000210031
:100118008E1220000E1E8D280E1A902821008E1691
:1001280003302000B300C3283108033A031D9E287A
:100138008422C3283108103A031DA5280030EC207A
:10014800C3283108113A031DAC280130EC20C3281C
:100158003108123A031DB3280230EC20C3283108B5
:10016800163A031DBA280630EC20C3283108173A7E
:10017800031DC1280730EC20C3280E1EC1280E1EFF
:10018800C828C3280E1EC6280E1ECD28C8280E1E35
:10019800CB280E1ED228CD280E1ED0280E1AD22803
:1001A800EE233308013A0319E328023A0319E52834
:1001B800073A0319E7280F3A0319E928EB2830080A
:1001C800FF293008422A3008C32A3008AB2B080020
:1001D800F500EE23082921000C1423000C14122921
:1001E80021008C1423008C14122921000C152300E3
:1001F8000C15122921000E1523000E1512292100B5
:100208008E1523008E151229750884000830040203
:10021800031812298331C9300407820021009E1770
:100228008F309E05FC309E057508F300F30DF30D25
:100238001D087306833973069D001D149D149D18AF
:100248002329BB234D23F400F4367408483A031DD0
:10025800462921008E1220000E1E2F290E1A32293F
:1002680021008E161B08FA2220000E1E38290E1AAD
:100278003B2921001C08FA2220000E1E40290E1ED0
:100288004929432920000E1E46290E1E0800492927
:10029800EE23A6217508AC007408AB007308AA0009
:1002A8007208A900BB234D232000A800A8362808FF
:1002B800483A031DA12921008E1220000E1E612933
:1002C8000E1A642921008E1620002908FA2220001F
:1002D8002A08A9002B08AA002C08AB00AC01AB1B0C
:1002E800AC030E1E75290E1A77292908FA22200058
:1002F8002A08A9002B08AA002C08AB00AC01AB1BEC
:10030800AC030E1E85290E1A87292908FA22200017
:100318002A08A9002B08AA002C08AB00AC01AB1BCB
:10032800AC030E1E95290E1A97292908FA222000D7
:100338000E1E9B290E1EA3299E290E1EA1290E1EE4
:100348000800A329A001A101A201A30122000C1207
:1003580089232000A401A501A601A70122000E14EB
:100368008923003020008E180130F600F701F801CB
:10037800F901A0047708A1047808A2047908A30465
:1003880024081F3A2504260427040319CF29A03579
:10039800A10DA20DA30D892322000E108923892304
:1003A8002000A40A0319A50A0319A60A0319A70A13
:1003B8002708803AFF0080307F02031DED290030B6
:1003C8002602031DED2900302502031DED292030EA
:1003D8002402031CB2298923892322000C168923AD
:1003E800892320002308F5002208F4002108F300DF
:1003F8002008F2000800F1000139F00021000C0883
:100408007006FE3970068C00F13671080139F0006B
:10041800F00D0C087006FD3970068C00F136710875
:100428000139F000F00DF00D0C087006FB3970066C
:100438008C00F1368C15F13671080139F000F00E98
:10044800F00D0C087006DF3970068C00F136710863
:100458000139F000F00DF00D0E087006FB3970063A
:100468008E00F13671080139F000F00DF00DF00D35
:100478000E087006F73970068E000800F100013981
:10048800F00022000C087006FE3970068C00F13668
:1004980071080139F000F00D0C087006FD3970067E
:1004A8008C00F13671080139F000F00DF00D0C08E0
:1004B8007006FB3970068C00F136F1367108013987
:1004C800F000F00EF00D0C087006DF3970068C0095
:1004D800F13671080139F000F00DF00D0E087006C4
:1004E800FB3970068E00F13671080139F000F00D05
:1004F800F00DF00D0E087006F73970068E00080032
:10050800EE23BB234D23F400F4367408483A031D48
:10051800BC2A21008E1220000E1E8F2A0E1A922A43
:1005280021008E16003020008E190130F500F535B7
:100538000E0C890C0139F504F5350C0E890C0139BE
:10054800F504F5350C0CF300F30C730C0139F504C4
:10055800F5350C0C890C0139F504F5350C0C01390D
:10056800F504F5350C080139F5047508FA22BF2A97
:1005780020000E1EBC2A20000E1E0800BF2AF10013
:100588000139F00024000C087006FE3970068C0052
:10059800F13671080139F000F00D0C087006FD39CC
:1005A80070068C00F13671080139F000F00DF00D7D
:1005B8000C087006FB3970068C00F1367108013999
:1005C800F000F00DF00DF00D0C087006F73970060C
:1005D8008C00F13671080139F000F00EF00D0C08AE
:1005E8007006DF3970068C00F1360800F100210032
:1005F8008E12F2010030F11B0130F000F00EF00D08
:1006080021000E087006DF3970068E00F1352000D3
:100618000E1E0B2B0E1A0E2B0830F20A7202031C48
:10062800FE2A21008E1608008B13151372089100FC
:100638007308F200F301F21BF303920015129516EA
:100648001515700893007108F000F101F01BF10313
:1006580094009512D923230015118B170800210047
:100668008C1624008C1620008C1A3D2BF030B2001A
:1006780008000730F001F1009A23F300FF3A031D48
:10068800492BA0302000B200080073082000B200F7
:1006980008000830F001F100F1080319612B20006F
:1006A8000E1E532B0E0E890C0139F0047103031D25
:1006B800F0350E1A5D2BF103502B7008080023004B
:1006C8008E018C0121000E168E1622000E128E123B
:1006D800D12321009513C03024008C0521008C16ED
:1006E80022008C1208008B137008230091007108F7
:1006F800F000F101F01BF103920015131516151502
:10070800D923230015118B170800F001F101F00A15
:100718000319F10A7108803AFF0080307F02031D37
:10072800972B0A307002031808008B2B70082300DF
:1007380091007108F000F101F01BF103920015130C
:1007480015140000000023001308F2000800F4004C
:100758000730F001F10077237408F0000730F10149
:10076800F201F300182374082000B20008002000EA
:100778008E1E8E1EBD2B8E1ABF2B0E1AC62B8E1ADE
:10078800BF2BC32B0E1E0800C62BEF28F428F92810
:10079800122912291229FE28032921008E140E106D
:1007A8000C1222000C168923892B55309600AA308A
:1007B8009600951400000000080078302100990484
:1007C800033099041A1A0800E62BE1236323332324
:1007D8000820EC2B0E1EEE2B8E1A0800EE2BB20111
:0607E800B3012000E92B23
:020000040001F9
:04000E00A4FFFFDD6F
:00000001FF
